:1000000019C030C02FC02EC02DC02CC03EC12AC088
:1000100029C028C027C026C025C024C00000000079
:1000200000FF00FF0000FFFFFF0000FF00FFFFFFD9
:1000300000FFFFFF11241FBE20E0A89521BD20E096
:1000400025BFE0EFF8E0A0E6B0E003C0C895319628
:100050000D92A036D9F7A0E6B0E001C01D92A837F6
:10006000E9F762C300C01895EF92FF920F931F93B8
:10007000F92FE82F972F862F042F152FE22EF32E1E
:10008000F8940024969587950794969587950794FC
:10009000982F802D2FEF30E0732F622F00D4972FF1
:1000A000862F80839183912F802F002496958795AA
:1000B0000794969587950794982F802D732F622F1C
:1000C000EED3972F862F828393839F2D8E2D00242E
:1000D000969587950794969587950794982F802DE8
:1000E000732F622FDCD3972F862F84839583789488
:1000F0001F910F91FF90EF900895CF92DF92EF92B2
:10010000FF920F931F93C82ED92EE62EF72E042FA1
:10011000152F312F202F5F2D4E2D7D2D6C2D82E63A
:1001200090E0A2DF312F202F5F2D4E2D7D2D6C2DE5
:1001300089E690E099DF312F202F5F2D4E2D7D2D08
:100140006C2D80E790E090DF1F910F91FF90EF9072
:10015000DF90CF90089580916800282F33278091F9
:100160006200909163002817390714F4C29801C007
:10017000C29A80916800282F332780916400909163
:1001800065002817390714F4C09801C0C09A8091FF
:100190006800282F33278091660090916700281708
:1001A000390714F4C19801C0C19A809168008F3357
:1001B00010F48F5F01C080E08093680080916F0031
:1001C000282F33278091690090916A0028173907FA
:1001D00014F4C59801C0C59A80916F00282F332769
:1001E00080916B0090916C002817390714F4C39824
:1001F00001C0C39A80916F00282F332780916D0032
:1002000090916E002817390714F4C49801C0C49A5D
:1002100080916F008F3310F48F5F01C080E0809376
:100220006F0080917600282F332780917000909185
:1002300071002817390714F4AA9801C0AA9A80916E
:100240007600282F33278091720090917300281731
:10025000390714F4A89801C0A89A80917600282F35
:10026000332780917400909175002817390714F492
:10027000A99801C0A99A809176008F3310F48F5FFE
:1002800001C080E08093760008951F920F920FB610
:100290000F9211242F933F934F935F936F937F930C
:1002A0008F939F93AF93BF93EF93FF938CE982BF9C
:1002B00080917700882351F0C29AC09AC19AC59A5A
:1002C000C39AC49AAA9AA89AA99A01C044DF81E065
:1002D00090E09093610080936000FF91EF91BF9157
:1002E000AF919F918F917F916F915F914F913F91CE
:1002F0002F910F900FBE0F901F9018958CE982BF21
:1003000082E083BF89B7826089BF0895482F592F43
:1003100014161506C4F420E030E001C088958091E1
:10032000600090916100892BC9F3109261001092D6
:1003300060002F5F3F4F2A3031058CF34150504011
:100340001416150644F308958827E19B83958823A6
:10035000D9F380E190E05FD299270895682F792F33
:100360008827E19B83958823D9F380E190E068D2C8
:1003700008958F929F92BF92CF92DF92EF92FF9259
:100380000F931F93CF93DF93882E992E20E030E0B8
:10039000532F422F6FEF70E080E790E065DE20E0A2
:1003A00030E0532F422F752F642F89E690E05CDEFA
:1003B00020E030E0532F422F752F642F82E690E02B
:1003C00053DE88EE93E0A2DF20E030E0532F422F8F
:1003D0006FEF70E089E690E047DE88EE93E096DF0D
:1003E00020E030E0532F422F6FEF70E082E690E084
:1003F0003BDE88EE93E08ADF20E830E04FEF50E00C
:1004000060E070E080E790E02FDE20E830E04FEF22
:1004100050E060E070E089E690E026DE20E830E021
:100420004FEF50E060E070E082E690E01DDE88EE85
:1004300093E06CDFEE24FF2404E610E0C8ECD0E08B
:100440000F2EF5E0BF2EF02D0F2EF3E0CF2EF02D66
:10045000DD246894D1F88B2D992787FD9095E80EBF
:10046000F91E8C2D992787FD9095080F191F8D2D4A
:10047000992787FD9095C80FD91FFF201CF4EE2403
:10048000FF240AC08FEFE816F10439F034F00F2E84
:10049000FFEFEF2EFF24F02DB194023311051CF471
:1004A00002E310E006C00F3F110521F01CF00FEF32
:1004B00010E0C194DD231CF4C0E0D0E006C0CF3FC3
:1004C000D10521F01CF0CFEFD0E0D1944C2F5D2F5F
:1004D000712F602F9F2D8E2D10DE8114910421F439
:1004E0008EE190E013DFB7CF1092770080E590E0C7
:1004F0000DDF81E08093770080E590E007DFABCFF0
:10050000DF91CF911F910F91FF90EF90DF90CF90EF
:10051000BF909F908F9008954F925F926F927F92BD
:100520008F929F92AF92BF92CF92DF92EF92FF9203
:100530000F931F93CF93DF93482E592EF72FE62F5B
:10054000B52DA42D8D919C916FEF70E096D1882EE2
:10055000992E97FCCF96882E992E082C892C000C6A
:10056000881C9908000C881C991CD52DC42D8A81E3
:100570009B816FEF70E081D1C82ED92ED7FCCF962A
:10058000C82ED92E0C2CCD2C000CCC1CDD08000C58
:10059000CC1CDD1CD52DC42D8C819D816FEF70E0AE
:1005A0006CD1D92FC82FD7FDCF96D92FC82F0C2E9D
:1005B000CD2F000CCC1FDD0B000CCC1FDD1F2E2F10
:1005C0003F2F220F331F2E0F3F1FF32FE22FE45E2A
:1005D000FF4FC895802D682E7724681879080FEF93
:1005E00010E0972D862D712F602F59D1662E772E12
:1005F000F32FE22FE35EFF4FC895802DA82EBB247A
:10060000AC18BD089B2D8A2D712F602F48D1A62EC6
:10061000B72EF32FE22FE25EFF4FC895802DE82E14
:10062000FF24EC1AFD0A9F2D8E2D712F602F37D1DC
:10063000E62EF72E01E010E081E090E067DE860C08
:10064000971CCA0CDB1CCE0DDF1D2C2F3D2F5D2D02
:100650004C2D792D682D952D842D06DD0F5F1F4FB4
:100660000F3F110549F344F3DF91CF911F910F9193
:10067000FF90EF90DF90CF90BF90AF909F908F90C2
:100680007F906F905F904F900895CF93DF93C1E07C
:10069000D0E06C2F7D2F82E690E03EDF6C2F7D2F27
:1006A00089E690E039DF6C2F7D2F80E790E034DF22
:1006B00067E070E082E690E02FDF67E070E089E6B7
:1006C00090E02ADF67E070E080E790E025DF88EEC9
:1006D00093E01CDE6C2F7D2F80E790E01DDF6C2FF8
:1006E0007D2F89E690E018DF6C2F7D2F82E690E069
:1006F00013DF67E070E080E790E00EDF67E070E016
:1007000089E690E009DF67E070E082E690E004DFD0
:1007100088EE93E0FBDD2196C730D1050CF4B9CF0C
:10072000B6CFDF91CF910895CFEDD0E0DEBFCDBF42
:100730008FEF88BB85BB82BBC29AC09AC19AC59A0B
:10074000C39AC49AAA9AA89AA99A8FE387BB84BB32
:100750008FEF81BB109261001092600010927700C1
:1007600040E050E0752F642F972F862FC6DCC6DD42
:1007700078948FEE05B6082205BE80E205B6082AF9
:1007800005BEE2DD8130910599F0823091051CF4BF
:10079000892B39F02FC08230910589F00397A1F0A1
:1007A00029C081E090E0DADD80E090E0E2DD30C059
:1007B00082E090E0D3DD81E090E0DBDD29C083E0E2
:1007C00090E0CCDD62DF24C08FEF90E0C7DD4FEF1B
:1007D00050E0752F642F972F862F8FDCC1E0109289
:1007E000770080E590E092DDC093770080E590E0AF
:1007F0008DDDF5CF80E090E0B1DD4FEF50E0752F5B
:10080000642F972F862F79DC8EE190E07FDDFCCF7F
:1008100080E090E0FFCFE199FECF9FBB8EBBE09AD6
:1008200099278DB30895E199FECF9FBB8EBBE09AC7
:1008300001960DB29FBB8EBBE09A802D9DB30895AB
:10084000E199FECF9FBB8EBB6DBB0FB6F894E29AC9
:10085000E19A0FBE08954115510571F0A82FB92FE7
:10086000E199FECF7FBB6EBBE09A6F5F7F4F0DB209
:100870000D9241505040B1F708955527002480FF54
:1008800002C0060E571F660F771F6115710521F014
:1008900096958795009799F7952F802D089597FB4A
:1008A000092E07260AD077FD04D00CD006D00020F0
:1008B0001AF4709561957F4F0895F6F7909581959C
:1008C0009F4F0895AA1BBB1B51E107C0AA1FBB1F66
:1008D000A617B70710F0A61BB70B881F991F5A95CC
:1008E000A9F780959095682F792F8A2F9B2F0895CF
:00000001FF
